:10000000DEFD9E00CEFCBC0000BCD1FFBCD07FBC9E
:10001000D9FFBCD800BCDC00BCD52EBCD451DD6FF0
:10002000DEEA9A8F9A019A8F9E01D0FFD105BC3CDF
:1000300037D437D837BC3D46BDD47BBDD47ABDEE6E
:100040007FBCEF11BDEF78BDEE7CBD4C7B3DCD9DFF
:10005000409C41BC42013DCD9D409C539D4192003E
:100060000492FF0A059D5392000CBD047D089D5328
:1000700092FF03BD047D9D4F9220010B3AB7BC4F08
:1000800000D908BC50000392FFF4BD047101E7BD24
:10009000046930A83F589D0394019C0392090220F3
:1000A00076BC030037B32076BD047220D3BD4C70FC
:1000B00020D3D22EDC37DE38BBA3C2FCBC0A009DA5
:1000C0000694019C069205010ABC0600BD04772F28
:1000D0009431548E00000000000000000000000079
:1000E0000000000000000000000000000000000010
:1000F0000000000000000000000000000000009C64
:10010000009DFE9C019DEF9C3BBDEF6D9D4F9200BD
:100110002E3F92012E4C92022E7392102E8E92112F
:100120002EA99D4F92200E92FF0B9D50A090019CF6
:100130005088BC4FFF21BEC005D0FABD04799D3B5D
:1001400095C0BDEF6FBDEF6EBDEF869CEF9D019C2E
:10015000FE9D008F9D0537A9BD04750B927E01079A
:10016000BD047FBC05008E50937321A49349011AEE
:1001700033869C07DB069D0735FCA39D0794019CF5
:1001800007CBF39D0594019C058E33869C07DB0607
:100190009D0734FCA39D0794019C07CBF39D059418
:1001A000019C058E33869C07DB069D07366CA39D5C
:1001B0000794019C07CBF39D0594019C058E9DF847
:1001C000920F010CD837BDD46BB8BDD47BBDD47AA7
:1001D0009DF89CFE9DD0977F9CD0AE967FBDD47934
:1001E0009CD0C8B8BDD469BDD46A213700000000D6
:1001F00000000000000000000000000000000000FF
:1002000000000000000000000000000000000000EE
:1002100000000000000000000000000000000000DE
:1002200000000000000000000000000000000000CE
:1002300000000000000000000000000000000000BE
:1002400000000000000000000000000000000000AE
:10025000000000000000000000000000000000009E
:10026000000000000000000000000000000000008E
:10027000000000000000000000000000000000007E
:10028000000000000000000000000000000000006E
:10029000000000000000000000000000000000005E
:1002A000000000000000000000000000000000004E
:1002B000000000000000000000000000000000003E
:1002C000000000000000000000000000000000002E
:1002D000000000000000000000000000000000001E
:1002E000000000000000000000000000000000000E
:1002F00000000000000000000000000000000000FE
:1003000000000000000000000000000000000000ED
:1003100000000000000000000000000000000000DD
:1003200000060C12181E242A30363C42484E545AFD
:1003300060666C72787E848A90969CA2A8AEB4BAED
:10034000C0C6CCD2D8DEE4EAF0F600060C12181EC5
:10035000242A30363C42484E545A60666C72787E8D
:10036000848A90969CA2A8AEB4BAC0C6CCD2D8DE7D
:10037000E4EAF0F600060C12181E242A30363C423D
:10038000484E545A6066A48E000000000000000031
:10039000000000000000000000000000000000005D
:1003A000000000000000000000000000000000004D
:1003B000000000000000000000000000000000003D
:1003C000000000000000000000000000000000002D
:1003D000000000000000000000000000000000001D
:1003E000000000000000000000000000000000000D
:1003F00000000000000000000000000000000000FD
:100400000000000000000000007D000000007000FF
:10041000700000147F147F1400122A7F2A240062C7
:1004200064081323003649350205000000700000FF
:10043000001C2241000000000041221C0022147F09
:1004400014220008083E0808000001060000000809
:10045000080808080000000100000002040810203D
:10046000003E4549513E0000217F010000234549DF
:100470004931004241495966000C14247F0400723E
:100480005151514E001E294949460040474850608D
:10049000003649494936003149494A3C00000014B8
:1004A00000000000011600000008142241000014A2
:1004B000141414140000412214080020404D502050
:1004C000003E415D4D39001F2444241F007F4949EF
:1004D0004936003E41414122007F4141413E007F7B
:1004E00049494941007F48484840003E414145272D
:1004F000007F0808087F0000417F4100A48E0000B3
:1005000000020101017E007F08142241007F0101E9
:100510000101007F2018207F007F1008047F003E2B
:100520004141413E007F48484830003E4145423D00
:10053000007F484C4A310032494949260040407FFB
:100540004040007E0101017E007C0201027C007FB0
:10055000020C027F0063140814630060100F106027
:10056000004345495161007F7F414141002010080F
:100570000402004141417F7F00040810080400018B
:100580000101010100004020100000021515150FA7
:10059000007F0911110E000E11111102000E111130
:1005A000097F000E1515150C00083F484020001863
:1005B0002525253E007F0810100F0000115F010067
:1005C000000201115E00007F040A11000000417F5B
:1005D0000100001F100C100F001F0810100F000E5C
:1005E0001111110E001F14141408000814140C1F0C
:1005F000001F08101008000915151502A48E000030
:1006000000107E110102001E0101021F001C0201E8
:10061000021C001E0106011E00110A040A11001826
:100620000505051E001113151911000008364100BB
:100630000000007F00000000413608000002551550
:10064000550F001E4101421F000E5111510E00FFB7
:10065000FFFFFFFF000008700000003F5252522CC5
:10066000001E4101411E000F5424540FA48E0000AF
:10067000000000000000000000000000000000007A
:10068000000000000000000000000000000000006A
:10069000000000000000000000000000000000005A
:1006A000000000000000000000000000000000004A
:1006B000000000000000000000000000000000003A
:1006C000000000000000000000000000000000002A
:1006D000000000000000000000000000000000001A
:1006E000000000000000000000000000000000000A
:1006F00000000000000000000000000000000000FA
:100700002A2A2A202D2D3E2044696573206973749E
:100710002065696E20426569737069656C20667535
:10072000657220496872656E2057657262657465EE
:1007300078742E203C2D2D2D2020576965206D6169
:100740006E2073696568742C207A696568656E200F
:100750004C61756673636872696674656E20426C7D
:1007600069636B6520617566207369636821202E5B
:100770002E2E2E2E2E2E2E456E747769636B656C91
:100780007420766F6E20574F484C52414245204CA2
:100790006963687473797374656D652E2E2E2E2EC1
:1007A0002E2E2E202A2A2A207EBD047501033C41CC
:1007B0008EA48EBD4C71282D9D4694019C469209B5
:1007C000022813BC46009D4794019C4792050228CD
:1007D00013BC47009D4894019C489209022813BC11
:1007E00048009D4994019C499205022813BC490088
:1007F0009D4A94019C4A920911920301169D4B92C5
:10080000020110BC4A00BC4B0009BC4A009D4B943D
:10081000019C4BBD4C7216BD4C700111BD4C710D4D
:100820009D4D94019C4D920F0103BD4C688E0000BC
:1008300000000000000000000000000000000000B8
:1008400000000000000000000000000000000000A8
:100850000000000000000000000000000000000098
:100860000000000000000000000000000000000088
:100870000000000000000000000000000000000078
:100880000000000000000000000000000000000068
:100890000000000000000000000000000000000058
:1008A0000000000000000000000000000000000048
:1008B0000000000000000000000000000000000038
:1008C0000000000000000000000000000000000028
:1008D0000000000000000000000000000000000018
:1008E0000000000000000000000000000000000008
:1008F00000000000000000000000000000000000F8
:10090000A48E2D0000000000000000000000000088
:100910000000003C00713100000079736177320003
:1009200000637864653433000020766674723500A5
:10093000006E6268677A360000006D6A75373800AD
:10094000002C6B696F303900002E2D6C8070830095
:1009500000007E237F0000000000002B000000004C
:1009600000000000000000000031003437000000EB
:100970003000323536382F00000033002B392A0082
:100980002D0000000000000000000000000000003A
:100990000000003E00512100000059534157220041
:1009A0000043584445240000002056465452250078
:1009B000004E4248475A260000004D4A552F280055
:1009C000003B4B494F3D2900003A5F4C00503F002F
:1009D00000008582846000000000002A0000000002
:1009E000000000000000000000310034370000006B
:1009F0003000323536380000000033002B392A0031
:100A0000BD4C71022A5A9D3E950F93092AA79C3E20
:100A10009D4E920001099D3E9C4BBC3C2F2A4E925C
:100A20000101099D3E9C4ABC3C232A4E9202010EC4
:100A30009D3E9C49BC3C1DBC4600BC4700109D3EF1
:100A40009C48BC3C35BC4E00BC4600BC47009D4E9B
:100A50009401920498009C4E2AA7BD0972022A8034
:100A6000BD096A9D3C92372AA7BC3E009CFE9D3E74
:100A700031689CFE940C9C3C3C9E3DE33FCD2AA5F6
:100A80009D3C9CFE9D3E31689CFE921301119D424F
:100A900092FF033AA8079D439201023AA898199C35
:100AA0003C3DE33C843C6D8ED506D22EDC37DE38EF
:100AB000BBA3C2FCC5F48ED600D908DE3A9D52A66F
:100AC000C901109D3AA0B09C3A89F59DF69401DECB
:100AD000F6A6EDBDF6700105BD5277058EBD5277C5
:100AE0008E9D52957F9C3E9D3E9301022C3A92082A
:100AF0000110BC4202BC43003FC4BD4C69BD046A46
:100B00002C3A92070116BD4C79BD4C78BD4C6BBC9C
:100B10004E00BD047A3FC4BC3C352C3A9217022BE0
:100B200046BD04722C3ABC4202BC43003FC4BD4CDB
:100B3000730105BD4C6B2C3ABD4C7BBD4C68BD4C64
:100B400069BD4C6A2C3A921F022B7ABD04721ABD01
:100B50004C7216BD4C7ABD4C78BD4C6BBC4E00BD82
:100B6000047A3FC4BC3C352C3ABD4C6ABD4C68BDD0
:100B7000046ABC4202BC43002C3ABD04722BA4920E
:100B80000F022C3ABD047ABD4C68BD4C69BC3D4691
:100B9000BC4202BC4300BC0500D437BC3C373FC458
:100BA0003C6D2C3A92660103BD097A925A022BFDE4
:100BB000BD046ABC4D00BD4C710105BD4C692C3AA9
:100BC0009D429301069D4393000104BD047D03BD36
:100BD000046D9D429C419D439C539D429C3EBD049F
:100BE0006BBD046CBC0500BC4200BC43003DE39DF2
:100BF000439C3EBC42013DE3BC42022C3A937F2C15
:100C00003A92590492120117BD4C702C3ABD0474EB
:100C10000107BD046C3C6D2C3ABD047C3C6D1BBDD2
:100C2000097201033A0013BD04740105924C029449
:100C30008039009200049C3E3A00BD096FBD046EED
:100C40008E3DCD9D53920001059D419202103C8442
:100C50009D42BD418201139D43BD5382010CBC42A4
:100C600002BC4300BD047FBC05009D408E9D3C9CA2
:100C7000FEBD04740103988102985F31689CFE9464
:100C8000069C3C8EA09D4290019C429D4390009CFE
:100C9000439D4392020106BC4301BC42FF8E9D422C
:100CA00094FF92FF010ABC42FF9D4394FF9C438E38
:100CB0009201039C428E9C429D439200BC42028E54
:100CC000DEEFDCE98E9D429C3FBC45013D438EBD7D
:100CD000D57CBDD46CBDD07FBDD47CBDD47DBDD40E
:100CE0006DBDD46CBDD47DBDD46DBDD47CBDD47D73
:100CF000BDD46DBD437003BDD46CBDD47DBDD46D7A
:100D0000BDD46C9D429CE9BDEF6ABDEE7BBDEF7A20
:100D1000BDEF72FC9D409CE9BDEF7ABDEF72FCBD5A
:100D2000D06FBDEE6BBDD07F3DC4BDD06F8EBDD04A
:100D30006FB8BDD07FB8B8BDD67601FBBDD06FBD52
:100D4000EE6B8EBDD57CBDD46CBDD07F6ABDEE7B15
:100D50009D43970C9CE97A72FE9D3FB67A72FEBD68
:100D6000457007BDD06FBDEE6B8EBD45712DBBBD0F
:100D700045722DC1BDEE6B64DA08BDD47DB8BDD41B
:100D80006DBDD6760102A101A0B0CAEEBDD06FBC88
:100D90004000B088BD407FB088BD407EB088BD4077
:100DA0007DB088BD407CB088BD407BB088BD407AB6
:100DB000B088BD4079B088BD40788E9D40B67A72CB
:100DC000FEBDD06FD712DAFFCAFEC7FA8E3CC0BD97
:100DD000EF683CC59D40BDD47CBDD56CBDEE6BBD00
:100DE000EF788E9D3E9C40BDEF683CC03E1F3CCFDF
:100DF0003DFFBDD47CBDD56CBDEE6BBDEF788EBD27
:100E0000D57CBDD46CBDD07F6ABCE908BDEE7B7AD1
:100E100072FEBCE9007A72FEBDD06FBDEE6B8EBD76
:100E2000D57CBDD46CBDD07F6ABCE909BDEE7B7AB0
:100E300072FEBCE9807A72FEBDD06FBDEE6B8EBDD6
:100E4000D6702122BC4F01BC50002122BDD67002B9
:100E50002122BD517605BD517E2122BD516E9D508E
:100E6000A1910A892ED6910A882ED6BC4F02BC5079
:100E7000012122BDD67021229D50A1910C892ED630
:100E8000910789022ED6BC4F10BC50002122BDD63E
:100E9000700221229D50A19101892ED69106882EA3
:100EA000D6BC4F11BC50002122BDD67021229D50CE
:100EB000A19101892ED6910489059102891802A079
:100EC00001A19D52B09C52BC5000C905BC4F2021CD
:100ED00022BC4F102122BC4FFF2122000000000045
:100EE0000000000000000000000000000000000002
:100EF00000000000000000000000000000000000F2
:100F00000E141A20262C32383E444A50A48E003E3D
:100F10004549513E0000217F0100002345494931E8
:100F2000004241495966000C14247F04007251515B
:100F3000514E001E2949494600404748506000363E
:100F400049494936003149494A3C00000014000033
:100F5000000000000000A48EBD4C70022F7F9D4B4E
:100F6000DE353F809D4A3F809D0393050103980B2A
:100F700002980A3F809D493F809D483F803FB68E42
:100F80003F0C9C07DB069D073F56A39D0794019CE1
:100F900007CBF38E55D2069A00C2FC9D0894019CA3
:100FA0000892070110BC0800BD046FBD4C7306BD5C
:100FB0004C78BC4D008EBD4C7101089D039305011A
:100FC000023C6D8ED52FDE389B00C5FC8E9D439272
:100FD00001069D429306018E9D42A191059C429D72
:100FE000439100D205BC3C373DCD9C3E3C849D3CAA
:100FF0009CFE9D3E31689CFE9C3CC2EC8E00000035
:00000001FF
